:020000040000FA
:0400000042EF03F0D8
:040008004EEF1BF0AC
:0800180079EF1BF0030B986F58
:10002000000EF76E280E07D0B9F9D9990F0B986F0B
:10003000000EF76E460EF66E9851F626D8B0F72AE7
:100040000800F55012003031323334353637383944
:10005000414243444546D0EC10F0BFEC00F0FDECCB
:100060001EF047C06FF006D0D0EC10F0BFEC00F0EF
:10007000140E6F6F6AEC21F0F4EC22F022C284F0CF
:1000800023C285F024C286F025C287F026C288F0FC
:100090008DEC26F0120022C284F023C285F024C227
:1000A00086F025C287F026C288F088AF12D0F0EC27
:1000B0001EF0846B856B866B876B886B84C036F211
:1000C00085C037F286C038F287C039F288C03AF26C
:1000D0001AD031C284F032C285F033C286F034C205
:1000E00087F035C288F0A8EC2AF084C036F285C0CB
:1000F00037F286C038F287C039F288C03AF2BFECD6
:1001000025F08FEC20F065C03BF066C03CF012009B
:1001100037C06FF038C070F063EC21F0E9EC22F0EA
:100120000EC289F00FC28AF010C28BF011C28CF09F
:1001300012C28DF0FFEC22F013C289F014C28AF0D3
:1001400015C28BF016C28CF017C28DF0C2EC23F0F2
:100150003BC289F03CC28AF03DC28BF03EC28CF0BB
:100160003FC28DF0C2EC23F084C027F285C028F294
:1001700086C029F287C02AF288C02BF2120035C04F
:100180006FF036C070F063EC21F0E9EC22F00EC2A3
:1001900089F00FC28AF010C28BF011C28CF012C22B
:1001A0008DF0FFEC22F013C289F014C28AF015C260
:1001B0008BF016C28CF017C28DF0C2EC23F03BC25C
:1001C00089F03CC28AF03DC28BF03EC28CF03FC247
:1001D0008DF0C2EC23F084C022F285C023F286C0E9
:1001E00024F287C025F288C026F2120039C06FF0D1
:1001F0003AC070F063EC21F0E9EC22F018C289F00B
:1002000019C28AF01AC28BF01BC28CF01CC28DF08E
:10021000FFEC22F01DC289F01EC28AF01FC28BF0D3
:1002200020C28CF021C28DF0C2EC23F03BC289F0D9
:100230003CC28AF03DC28BF03EC28CF03FC28DF0D2
:10024000C2EC23F084C02CF285C02DF286C02EF2C1
:1002500087C02FF288C030F2120022C284F023C27D
:1002600085F024C286F025C287F026C288F088AFC8
:1002700013D085EC25F089C031F28AC032F28BC0F0
:1002800033F28CC034F28DC035F2F0EC1EF065C054
:100290008AF166C08BF128D022C284F023C285F097
:1002A00024C286F025C287F026C288F02CC289F0CD
:1002B0002DC28AF02EC28BF02FC28CF030C28DF08E
:1002C000BCEC23F084C031F285C032F286C033F238
:1002D00087C034F288C035F2BFEC25F08FEC20F0F7
:1002E00065C08AF166C08BF11200000EF86E380E00
:1002F000F76E8A0EF66EA9EC12F022C284F023C2C9
:1003000085F024C286F025C287F026C288F069EC09
:1003100029F0030E8E6F010E8F6F91850BEC29F083
:100320005CEF28F0140E91EC12F0FDEC1EF08AC187
:100330006FF08BC170F051EC29F0040E8E6F8F6B53
:1003400030EF28F0000EF86E380EF76E8E0EF66E57
:10035000A9EC12F031C284F032C285F033C286F0CB
:1003600034C287F035C288F069EC29F0040E8E6F34
:10037000020E8F6F0BEC29F05CEF28F0000EF86E88
:10038000380EF76E940EF66EA9EC12F036C284F0B9
:1003900037C285F038C286F039C287F03AC288F099
:1003A00069EC29F0040E8E6F020E8F6F0BEC29F0B2
:1003B0005CEF28F0140E91EC12F036509DEC12F028
:1003C00035509DEC12F093EC12F03A509DEC12F087
:1003D00039509DEC12F012000EEC02F0D0EC02F05D
:1003E00075EC01F0A2EC01F0A6EC02F0120000EEB8
:1003F00014F0E950125C946F610E91EC12F094537A
:100400000AE0060E946107D0EE50300908EC12F0B5
:10041000942FFAD702D09FEC1BF01200000EF86E5A
:10042000380EF76E7A0EF66EA9EC12F0EFEC1EF0B5
:100430001EC06FF01FC070F051EC29F0030E8E6FDC
:1004400030EC28F0000EF86E380EF76E7E0EF66E69
:10045000A9EC12F0EFEC1EF01DC06FF051EC29F08A
:10046000030E8E6F30EC28F01C6610D0000EF86E74
:10047000380EF76E9A0EF66EA9EC12F0000EF86EBA
:10048000380EF76EA00EF66EA9EC12F0010E1C628B
:1004900010D0000EF86E380EF76EA60EF66EA9ECB0
:1004A00012F0000EF86E380EF76EAC0EF66EA9EC78
:1004B00012F0020E1C6210D0000EF86E380EF76EAD
:1004C000B20EF66EA9EC12F0000EF86E380EF76E52
:1004D000B80EF66EA9EC12F0030E1C6210D0000EDE
:1004E000F86E380EF76EBE0EF66EA9EC12F0000E26
:1004F000F86E380EF76EC40EF66EA9EC12F0040E0C
:100500001C6210D0000EF86E380EF76ECA0EF66E32
:10051000A9EC12F0000EF86E380EF76ED00EF66EE3
:10052000A9EC12F0050E1C6210D0000EF86E380E09
:10053000F76ED60EF66EA9EC12F0000EF86E380EBD
:10054000F76EDC0EF66EA9EC12F01200000EF86EDB
:10055000380EF76E860EF66EA9EC12F05150300987
:1005600008EC12F03A0E08EC12F0EFEC1EF07AC133
:100570006FF07BC170F00A0E746FF1EC26F051EC55
:1005800029F0050E8E6F030E8F6F30EC28F0000EF1
:10059000F86E380EF76EE60EF66EAFEC12F0120043
:1005A000000EF86E380EF76EE20EF66EA9EC12F041
:1005B00045C0E8FF300908EF12F0F29E6F6F080E99
:1005C000946F83885DEC11F05FEC11F06F33D8A06D
:1005D00005D083885FEC11F0839804D083985FEC9A
:1005E00011F083885FEC11F0942FF0D783985DECC5
:1005F00011F0F28E1200756F741B7551DED7746B9B
:10060000AA0EF9DFAA0EF7DF45C0E8FFF4DF1CC031
:10061000E8FFF1DF1DC0E8FFEEDF1EC0E8FFEBDF03
:100620001FC0E8FFE8DF8CC1E8FFE5DF8DC1E8FF10
:10063000E2DF27C2E8FFDFDF28C2E8FFDCDF29C2F4
:10064000E8FFD9DF2AC2E8FFD6DF2BC2E8FFD3DFFD
:100650007AC1E8FFD0DF7BC1E8FFCDDF51C0E8FF02
:10066000CADFCC0EC8DF7451A8DF12000B0E116276
:1006700003D00A0E116E05D00A0E116202D00B0EC5
:10068000116E120070EC11F0B5EC07F0FDEC10F0FB
:100690000DEC11F0EDEC10F02DEC11F01BEC1BF05B
:1006A00035EC11F01DEC11F001017A6B7B6B7C6B6A
:1006B0007D6B7E6B7F6B806B816B826B836B846BDE
:1006C000856B0001BEEC11F00C6A3EEC08F000EE08
:1006D00014F0E9CF12F0EACF13F00794ECEC01F03C
:1006E000448C80A60AD084EC0BF049EC11F0B9ECF4
:1006F0000BF049EC11F089EC12F0D0EC10F0365010
:10070000385C02E13550375CD8B004D035C037F0E2
:1007100036C038F05DEC05F007A20CD0A3EC14F065
:10072000079281B0FED78250F00BE838116E36EC9C
:1007300003F010D0B8EC12F0D8A05ED0D1EC12F0DB
:10074000110E116202D0C4EC04F0120E116202D03C
:10075000FDEC04F007B43FD0070E116205D01D6612
:100760001D06B9EC07F047D00A0E116206D0FF0E45
:100770001D621D2AB9EC07F03ED0060E11620DD0A5
:100780001F5202E11E5208E01E061E28D8B41F06A2
:10079000D8B41E52B9EC07F02ED0090E116211D058
:1007A000820E6F6F030E706F1F50705D02E11E505E
:1007B0006F5DD8A005D01E2AD8B41F2AB9EC07F067
:1007C0001AD0080E116207D01C2A060E1C601C6A83
:1007D000B9EC07F010D007840C0E116205D0AFEC15
:1007E00005F017EC06F005D0AFEC05F002E317ECCE
:1007F00006F0F7EC01F0116A07AA0BD02BEC00F021
:1008000006E2426606D0B9EC07F0079A02D0640E01
:10081000426E444E448C010E446204D00EEC02F051
:10082000D0EC02F0020E446202D075EC01F0030E2F
:10083000446215D07AC16FF07BC170F07CC174F056
:100840007DC175F07551705D02E174516F5DD8B472
:1008500006D0F6EC17F07AC17CF17BC17DF1040E75
:10086000446202D0A2EC01F0050E446202D0BEEC5C
:1008700001F0060E446202D0A6EC02F0070E4462BC
:1008800000D0080E446200D0090E44620CD01E0E47
:1008900091EC12F0415204E1405202E1200E01D0ED
:1008A0002A0E08EC12F00A0E446200D00B0E4462CD
:1008B0001AD04BEC00F03C6603D03B6601D009D067
:1008C0003BC08CF13CC08DF1E00E406E2E0E416EAF
:1008D0000AD0415208E1405206E101018C6B8D6B58
:1008E0000001376A386A0C0E446200D00D0E446273
:1008F00000D00E0E446208D0BFEC00F088EC00F08F
:10090000F6EC00F02DEC01F00F0E446208D04650DA
:10091000455CD8B404D045C046F0F6EC17F0100E94
:10092000446221D051A21FD082C16FF083C170F008
:1009300084C174F085C175F07551705D02E1745128
:100940006F5DD8B410D082C17AF183C17BF182C1CE
:1009500084F183C185F182C17EF183C17FF17EC1C3
:1009600080F17FC181F1110E446200D0120E446209
:1009700006D007AC04D0436602D0079C8398130EC0
:10098000446200D07DEF03F089EC12F0000EF86EA7
:100990003A0EF76E580EF66EA9EC12F0000EF86ED5
:1009A0003A0EF76E6E0EF66EA9EC12F0000EF86EAF
:1009B0003A0EF76E840EF66EA9EC12F03BEC13F0D3
:1009C0004BEC11F034EC13F0D1EC12F0010E11628B
:1009D00002D024EC0AF0020E116202D01DEC09F0E4
:1009E000030E116202D040EC0DF0040E116202D031
:1009F000BFEC0DF089EC12F0120089EC12F0000E41
:100A0000F86E3A0EF76E580EF66EA9EC12F0000E64
:100A1000F86E3A0EF76E9A0EF66EA9EC12F0000E12
:100A2000F86E3A0EF76EB00EF66EA9EC12F03BECD3
:100A300013F04BEC11F034EC13F0D1EC12F0010E8A
:100A4000116202D03EEC0EF0020E116202D085EC73
:100A50000FF089EC12F0120036EC05F03F6604D07E
:100A60003E6602D0D8901200D88012009382B80E51
:100A7000946FD66A3E6A1AEC08F0942FFCD70000F7
:100A800000003F6A93928A82D650D8A4D6BC58EF11
:100A900005F03F6E8A923E060BE0D6503F5C8A829C
:100AA000F9E0D8903F323E32D8903F323E3202D009
:100AB0003E6A3F6A93828A82120034EC00F045E37A
:100AC000A3EC14F051B209D051A007D05BEC11F0A7
:100AD0007EC16FF07FC170F03AD0050E966F716BDA
:100AE0002CEC05F032E33EC06FF03FC070F036EC06
:100AF00005F03F50705D02E13E506F5DD8B41DD0EF
:100B00006F2BD8B4702B3F50705D02E13E506F5D8B
:100B1000D8B413D06F076F29D8B47007D8B46F5307
:100B20006F076F29D8B47007D8B46F533F50705D0A
:100B300002E13E506F5DD8A405D0712B030E7163A6
:100B400002D005D0716B962FCBD7D89007D06FC04D
:100B500082F170C083F1A3EC14F0D8801200190E5A
:100B6000125C10E012C0E9FF13C0EAFF0B0E116225
:100B700001D0116A11C0EEFFE9CF12F0EACF13F0F5
:100B8000D89003D00C0E196ED8801200EFEC1EF036
:100B90000C0E195C09E1030E146E18C065F017C045
:100BA00066F016C067F011D00C0E185C07E1020E5B
:100BB000146E17C065F016C066F007D00C0E175CF7
:100BC0000DE1010E146E16C065F01EEC2AF04FEC1C
:100BD00022F065C01AF066C01BF01200146AF0EC37
:100BE0001EF065C01AF066C01BF012000054657359
:100BF00074706D696E20202020202020202020206D
:100C0000200000773430393420202020202020207C
:100C1000202020202020200000526561646D656D39
:100C20006F72792046414C53452020202000040E4D
:100C300014605FD00C0E155C0AE00C0E165C07E029
:100C40000C0E175C04E00C0E185C01E002D080EF83
:100C500007F0190E125CD8A48FEF07F0EFEC1EF02E
:100C600018C065F017C066F016C067F015C068F0D0
:100C700014C069F01EEC2AF04FEC22F0F7EC1FF0E4
:100C800004EC1FF00A0E746F65EC27F06FC07EF164
:100C900070C07FF151A02CD07EC16FF07FC170F089
:100CA00080C174F081C175F07551705D02E17451BD
:100CB0006F5DD8B41DD07EC17AF17FC17BF17EC15A
:100CC00080F17FC181F17EC182F17FC183F182C158
:100CD00084F183C185F1F6EC17F007AA09D02BEC5B
:100CE00000F004E2B9EC07F0079A02D0640E426EFD
:100CF00007D1143A15501412400E146203D09CEC24
:100D000007F0FED0410E146217D0C6EC05F0010EBC
:100D1000146212D0050E6F6F000E706F1B50705D65
:100D200002E11A506F5DD8B002D0050E1A6E1AC0DB
:100D30001CF0B9EC07F0E4D0420E146215D0C6ECFA
:100D400005F0145211E0FF0E6F6F000E706F1B5014
:100D5000705D02E11A506F5DD8B001D01A681AC0F8
:100D60001DF0B9EC07F0CCD0430E14621AD0C6ECDB
:100D700005F0145216E0830E6F6F030E706F1B5058
:100D8000705D02E11A506F5DD8B004D0830E1A6E08
:100D9000030E1B6E1AC01EF01BC01FF0B9EC07F04B
:100DA000AFD0440E146216D0C6EC05F0010E1462EA
:100DB00011D01AC045F0010E456002D0010E456EFB
:100DC000050E456402D0050E456E25EC11F01BECB6
:100DD0001BF096D0450E146205D0C6EC05F06EEC03
:100DE00017F08ED0460E14620DD0C6EC05F01466D6
:100DF00003D06EEC18F084D0010E146203D004EC22
:100E000018F07ED0490E146203D074EC16F078D03E
:100E1000510E146208D0C6EC05F0010E146203D026
:100E200006EC16F06DD0520E146204D043EC16F0AE
:100E3000466866D0530E146222D0C6EC05F0010E4F
:100E400014621DD01AC06FF06F6703D05192519099
:100E500013D0010E6F6303D0519251800DD0020E5A
:100E60006F6303D05182519007D0030E6F6303D09C
:100E70005182518001D003D03DEC11F041D0540E8D
:100E8000146216D0C6EC05F0146603D095EC07F09A
:100E900037D0010E14620CD0090E1A6203D09AECFE
:100EA00017F02ED0070E1A6203D0B5EC17F028D039
:100EB000560E14620DD080B608D0C6EC05F0020EB6
:100EC00014621ED090EC07F01BD0A6EC08F018D0EE
:100ED000570E146203D04EEC14F012D0580E146268
:100EE00005D055EC11F0FFEC02F00AD0590E146257
:100EF00007D015EC1BF085EC08F01BEC1BF000D0C4
:100F000089EC12F0146A156A166A176A186A196A67
:100F100000EE14F0E9CF12F0EACF13F007941200BC
:100F20001AC047F015EC11F012008388640E436E6E
:100F3000078C406A416A12001D6A1C6A1E6A1F6A99
:100F400001017A6B7B6B7C6B7D6B7E6B7F6B806B47
:100F5000816B826B836B846B856B00013EEC08F0C8
:100F6000B5EC07F095EC07F012008388326A336A1B
:100F700043D083881DC032F0336AEFEC1EF01EC0F0
:100F80006FF01FC070F0640E746F000E756F65EC2B
:100F900027F0655308E03388650765B1338E65B384
:100FA000338C65B5338A74C00FF00E500F5CD8A433
:100FB000F4EC08F01C5220E0010E1C6202D03382D7
:100FC0001BD0020E1C6202D0338416D0030E1C62AA
:100FD00004D03382338433860FD0040E1C6204D0D5
:100FE00033823384338008D0050E1C6205D03382EF
:100FF00033843386338000D0100E986F8C9C32324D
:101000003332D8B08C8C17EC08F08C8E17EC08F0CB
:101010008C9E982FF3D78C8A13EC08F08C9A5BEC9B
:1010200011F0839812000000000000000000000092
:101030000000000000000000000012001E0E0D6EF7
:10104000818E0C500EEC00F08A6E5BEF11F05BECC1
:1010500011F0819E12000D5064EF11F00C2A040E65
:101060000C600C6A12000C06FF0E0C6202D0030E1C
:101070000C6E1200040E0D620D061200838889ECBE
:1010800012F0000EF86E370EF76EE00EF66EA9EC59
:1010900012F0000EF86E380EF76E380EF66EA9ECF0
:1010A00012F01EEC08F0D20E976F80A40FD02EEC39
:1010B00008F00C500EEC00F08A6E2BEC08F03AECC5
:1010C00008F080A403D0972FF2D70ED027EC08F0B9
:1010D000000EF86E380EF76E4E0EF66EA9EC12F09A
:1010E0000E6A0F6A83980CD027EC08F0000EF86E99
:1010F000380EF76E640EF66EA9EC12F045EC11F0A6
:101100004BEC11F089EC12F0120080B612001CC0FA
:1011100086F11DC087F11EC088F11FC089F11C6ACD
:101120001D6A1E6A1F6AECEC01F0B9EC07F08388B7
:10113000079203008398079286C11CF087C11DF0B7
:1011400088C11EF089C11FF0B9EF07F083880792AC
:10115000079889EC12F0000EF86E370EF76EE00E6D
:10116000F66EA9EC12F0000EF86E370EF76EF60E62
:10117000F66EA9EC12F0000EF86E380EF76E0C0E3B
:10118000F66EA9EC12F01EEC08F02EEC08F00C50F4
:101190000EEC00F08A6E2BEC08F03AEC08F0B8EC9C
:1011A00012F0F3E30798079227EC08F0839889EC94
:1011B00012F0000EF86E370EF76EE00EF66EA9EC28
:1011C00012F0000EF86E370EF76EF60EF66EA9EC02
:1011D00012F0000EF86E380EF76E220EF66EA9ECC5
:1011E00012F04BEC11F0FF001EEC08F00E500F5CFB
:1011F0001FE0E8CF97F097BF0DD02EEC08F00C5011
:101200000EEC00F08A6E2BEC08F03AEC08F0972F09
:10121000F4D70ED0971F972B33EC08F00C500EEC40
:1012200000F08A6E2BEC08F03AEC08F0972FF4D718
:1012300027EC08F00FC00EF0120018C240F219C2DD
:1012400041F21AC242F21BC243F21CC244F21DC256
:1012500045F21EC246F21FC247F220C248F221C226
:1012600049F289EC12F0000EF86E3B0EF76E3E0E5E
:10127000F66EA9EC12F0000EF86E390EF76EA40EA1
:10128000F66EA9EC12F08BDBB8EC12F0FCE3D1ECBB
:1012900012F00C0E116201D0ABD0030E1162A8D077
:1012A00005C284F006C285F007C286F008C287F046
:1012B00009C288F08FEC20F065C00AF266C00BF21C
:1012C00089EC12F0000EF86E3B0EF76E540EF66EBF
:1012D000A9EC12F0000EF86E390EF76EA40EF66E41
:1012E000A9EC12F05CDBB8EC12F0FCE3D1EC12F0EC
:1012F0000C0E116201D07CD0030E116279D005C2B0
:1013000084F006C285F007C286F008C287F009C2E1
:1013100088F08FEC20F065C00CF266C00DF289EC0D
:1013200012F0000EF86E3B0EF76EAC0EF66EA9ECE6
:1013300012F07FDB84C018F285C019F286C01AF261
:1013400087C01BF288C01CF295DB84C01DF285C0EB
:101350001EF286C01FF287C020F288C021F240DB57
:1013600049EC11F0000EF86E390EF76EBA0EF66EFB
:10137000A9EC12F0D1EC12F089EC12F0FAD949EC98
:1013800011F0000EF86E390EF76EA40EF66EA9EC91
:1013900012F0D1EC12F00C0E116201D029D0030E24
:1013A000116226D089EC12F0000EF86E390EF76E3D
:1013B000360EF66EA9EC12F0000EF86E390EF76ECE
:1013C0004C0EF66EA9EC12F005EC11F049EC11F0A0
:1013D00089EC12F003DA49EC11F0000EF86E390EC8
:1013E000F76EBA0EF66EA9EC12F0D1EC12F02AD01C
:1013F00089EC12F0000EF86E390EF76E620EF66E82
:10140000A9EC12F0000EF86E390EF76E780EF66E3B
:10141000A9EC12F049EC11F089EC12F040C218F27C
:1014200041C219F242C21AF243C21BF244C21CF278
:1014300045C21DF246C21EF247C21FF248C220F248
:1014400049C221F2116A12000EC240F20FC241F2EB
:1014500010C242F211C243F212C244F213C245F268
:1014600014C246F215C247F216C248F217C249F238
:1014700089EC12F0000EF86E3B0EF76E3E0EF66E23
:10148000A9EC12F0000EF86E390EF76EA40EF66E8F
:10149000A9EC12F063DAB8EC12F0FCE3D1EC12F034
:1014A0000C0E116201D0ABD0030E1162A8D000C2A5
:1014B00084F001C285F002C286F003C287F004C244
:1014C00088F08FEC20F065C00AF266C00BF289EC60
:1014D00012F0000EF86E3B0EF76E540EF66EA9EC8D
:1014E00012F0000EF86E390EF76EA40EF66EA9EC2F
:1014F00012F034DAB8EC12F0FCE3D1EC12F00C0E7E
:10150000116201D07CD0030E116279D000C284F048
:1015100001C285F002C286F003C287F004C288F0DF
:101520008FEC20F065C00CF266C00DF289EC12F071
:10153000000EF86E3B0EF76E960EF66EA9EC12F0EA
:1015400078DA84C00EF285C00FF286C010F287C030
:1015500011F288C012F28EDA84C013F285C014F240
:1015600086C015F287C016F288C017F239DA49EC46
:1015700011F0000EF86E390EF76EBA0EF66EA9EC89
:1015800012F0D1EC12F089EC12F0BED849EC11F057
:10159000000EF86E390EF76EA40EF66EA9EC12F07E
:1015A000D1EC12F00C0E116201D029D0030E1162A1
:1015B00026D089EC12F0000EF86E390EF76E360E5A
:1015C000F66EA9EC12F0000EF86E390EF76E4C0EA6
:1015D000F66EA9EC12F0F5EC10F049EC11F089EC84
:1015E00012F047D949EC11F0000EF86E390EF76E83
:1015F000BA0EF66EA9EC12F0D1EC12F02AD089ECFA
:1016000012F0000EF86E390EF76E620EF66EA9EC4F
:1016100012F0000EF86E390EF76E780EF66EA9EC29
:1016200012F049EC11F089EC12F040C20EF241C206
:101630000FF242C210F243C211F244C212F245C28A
:1016400013F246C214F247C215F248C216F249C25A
:1016500017F2116A1200410E8D6F896B8A6B8B6BCA
:101660008C6B1200410E8D6F100E8C6F896B8A6B24
:101670008B6B120000C284F001C285F002C286F0BA
:1016800003C287F004C288F0E6DFFFEC22F035C029
:101690006FF036C070F063EC21F0F4EC22F0C2EC95
:1016A00023F0E0DF7FEC23F084C000F285C001F27C
:1016B00086C002F287C003F288C004F2120005C29D
:1016C00084F006C285F007C286F008C287F009C21E
:1016D00088F0C1DFFFEC22F039C06FF03AC070F043
:1016E00063EC21F0F4EC22F0C2EC23F0BBDF7FECE2
:1016F00023F084C005F285C006F286C007F287C0D9
:1017000008F288C009F21200000EF86E3B0EF76E68
:10171000960EF66EA9EC12F0000EF86E3B0EF76E08
:10172000C20EF66EA9EC12F00EC284F00FC285F064
:1017300010C286F011C287F012C288F0B2EC29F014
:10174000DAEC29F0000EF86E3B0EF76EC80EF66E5E
:10175000A9EC12F013C284F014C285F015C286F011
:1017600016C287F017C288F0B2EC29F0DAEC29F043
:101770001200000EF86E3B0EF76EAC0EF66EA9EC82
:1017800012F0000EF86E3B0EF76EC20EF66EA9EC6C
:1017900012F018C284F019C285F01AC286F01BC27A
:1017A00087F01CC288F0B2EC29F0DAEC29F0000EC8
:1017B000F86E3B0EF76EC80EF66EA9EC12F01DC265
:1017C00084F01EC285F01FC286F020C287F021C2BD
:1017D00088F0B2EC29F0DAEC29F01200000EF86E75
:1017E0003B0EF76EAC0EF66EA9EC12F0000EF86E22
:1017F0003B0EF76EC20EF66EA9EC12F018C26FF037
:1018000019C270F01AC271F01BC272F01CC273F0E0
:1018100073519DEC12F072519DEC12F071519DECE0
:1018200012F070519DEC12F06F519DEC12F0000E11
:10183000F86E3B0EF76EC80EF66EA9EC12F01DC2E4
:101840006FF01EC270F01FC271F020C272F021C290
:1018500073F073519DEC12F072519DEC12F07151C6
:101860009DEC12F070519DEC12F06F519DEC12F056
:101870001200000EF86E3B0EF76E960EF66EA9EC97
:1018800012F0000EF86E3B0EF76EC20EF66EA9EC6B
:1018900012F00EC26FF00FC270F010C271F011C2E0
:1018A00072F012C273F073519DEC12F072519DEC04
:1018B00012F071519DEC12F070519DEC12F06F51CD
:1018C0009DEC12F0000EF86E3B0EF76EC80EF66E31
:1018D000A9EC12F013C26FF014C270F015C271F0CF
:1018E00016C272F017C273F073519DEC12F0725170
:1018F0009DEC12F071519DEC12F070519DEC12F0C4
:101900006F519DEC12F01200FDEC1EF0000EF86E0F
:101910003B0EF76E260EF66EA9EC12F035C06FF096
:1019200036C070F051EC29F0040E8E6F30EC28F0C8
:101930001200FDEC1EF0000EF86E3B0EF76E320E3C
:10194000F66EA9EC12F039C06FF03AC070F051ECAD
:1019500029F0040E8E6F30EC28F0120055EC11F0D7
:10196000D0EC10F03AEC0BF0000EF86E3B0EF76E78
:101970000E0EF66EA9EC12F000C284F001C285F0E2
:1019800002C286F003C287F004C288F069EC29F035
:10199000050E8E6F8F6B0BEC29F05CEF28F055EC89
:1019A00011F0D0EC10F05FEC0BF0000EF86E3B0E77
:1019B000F76E1A0EF66EA9EC12F005C284F006C29C
:1019C00085F007C286F008C287F009C288F069EC8A
:1019D00029F0050E8E6F8F6B0BEC29F05CEF28F071
:1019E000000EF86E3B0EF76ECE0EF66EA9EC12F0FE
:1019F000FDEC1EF00AC26FF00BC270F051EC29F042
:101A0000040E8E6F30EC28F0000EF86E3B0EF76E71
:101A1000DA0EF66EA9EC12F0FDEC1EF00CC26FF0BF
:101A20000DC270F051EC29F0040E8E6F30EC28F0EE
:101A300012000AC26FF00BC270F063EC21F0E9EC07
:101A400022F0C0EC1FF00CC26FF00DC270F063EC1E
:101A500021F0F4EC22F0BCEC23F03CEC1FF01E0E65
:101A60006F6F6AEC21F0E9EC22F010EC1FF07FECD4
:101A700023F0120052EC1FF0FFEC22F0887F1200DE
:101A800013C284F014C285F015C286F016C287F026
:101A900017C288F00EC289F00FC28AF010C28BF014
:101AA00011C28CF012C28DF07FEC23F0887F8FEC96
:101AB00020F065C00AF266C00BF213C284F014C2B3
:101AC00085F015C286F016C287F017C288F01E0E88
:101AD0006F6F6AEC21F0F4EC22F0C2EC23F00EC23E
:101AE00089F00FC28AF010C28BF011C28CF012C2C2
:101AF0008DF07FEC23F0887F8FEC20F065C00CF236
:101B000066C00DF289EC12F0000EF86E3B0EF76E17
:101B1000960EF66EA9EC12F0F0EC0CF049EC11F018
:101B2000000EF86E390EF76EBA0EF66EA9EC12F0D2
:101B3000D1EC12F089EC12F084EC0BF049EC11F0CE
:101B4000000EF86E390EF76EBA0EF66EA9EC12F0B2
:101B5000D1EC12F089EC12F039EC0CF049EC11F0F8
:101B6000000EF86E390EF76EBA0EF66EA9EC12F092
:101B7000D1EC12F089EC12F00C0E116E12001DC2A5
:101B800084F01EC285F01FC286F020C287F021C2F9
:101B900088F018C289F019C28AF01AC28BF01BC2F1
:101BA0008CF01CC28DF07FEC23F0887F8FEC20F04E
:101BB00065C00AF266C00BF21DC284F01EC285F039
:101BC0001FC286F020C287F021C288F01E0E6F6F00
:101BD0006AEC21F0F4EC22F0C2EC23F018C289F098
:101BE00019C28AF01AC28BF01BC28CF01CC28DF095
:101BF0007FEC23F0887F8FEC20F065C00CF266C08C
:101C00000DF289EC12F0000EF86E3B0EF76EAC0E82
:101C1000F66EA9EC12F0F0EC0CF049EC11F0000EAD
:101C2000F86E390EF76EBA0EF66EA9EC12F0D1EC22
:101C300012F089EC12F0B9EC0BF049EC11F0000E47
:101C4000F86E390EF76EBA0EF66EA9EC12F0D1EC02
:101C500012F089EC12F0EEEC0BF049EC11F0000EF2
:101C6000F86E390EF76EBA0EF66EA9EC12F0D1ECE2
:101C700012F089EC12F00C0E116E12000EC240F23E
:101C80000FC241F210C242F211C243F212C244F238
:101C900013C245F214C246F215C247F216C248F208
:101CA00017C249F289EC12F0000EF86E3B0EF76E87
:101CB0006A0EF66EA9EC12F0000EF86E390EF76E91
:101CC000D00EF66EA9EC12F0146A156A166A176A3D
:101CD000186A356A366A18DEB8EC12F0FDE3D1EC0A
:101CE00012F00A0E116201D0E2D00C0E116205D082
:101CF00035C00AF236C00BF223D00B0E116201D0B0
:101D0000116A300E111216C017F015C016F014C06B
:101D100015F011C014F0EFEC1EF014C065F015C002
:101D200066F016C067F017C068F018C069F01EECC6
:101D30002AF04FEC22F065C035F066C036F0CBD704
:101D400089EC12F0000EF86E3B0EF76E800EF66E08
:101D5000A9EC12F0000EF86E390EF76ED00EF66E8A
:101D6000A9EC12F0146A156A166A176A186A356ABD
:101D7000366ACADDB8EC12F0FDE3D1EC12F00A0EBF
:101D8000116201D094D00C0E116205D035C00CF256
:101D900036C00DF223D00B0E116201D0116A300E45
:101DA000111216C017F015C016F014C015F011C0AE
:101DB00014F0EFEC1EF014C065F015C066F016C00C
:101DC00067F017C068F018C069F01EEC2AF04FECFD
:101DD00022F065C035F066C036F0CBD789EC12F042
:101DE000000EF86E3B0EF76E960EF66EA9EC12F032
:101DF00020DE84C00EF285C00FF286C010F287C0CC
:101E000011F288C012F236DE84C013F285C014F2DB
:101E100086C015F287C016F288C017F2E1DD49ECE2
:101E200011F0000EF86E390EF76EBA0EF66EA9ECD0
:101E300012F0D1EC12F089EC12F066DC49EC11F0F2
:101E4000000EF86E390EF76ED00EF66EA9EC12F099
:101E5000D1EC12F00A0E116201D029D00C0E1162E1
:101E600026D089EC12F0000EF86E390EF76E360EA1
:101E7000F66EA9EC12F0000EF86E390EF76E4C0EED
:101E8000F66EA9EC12F0F5EC10F049EC11F089ECCB
:101E900012F0EFDC49EC11F0000EF86E390EF76E1F
:101EA000BA0EF66EA9EC12F0D1EC12F02AD089EC41
:101EB00012F0000EF86E390EF76E620EF66EA9EC97
:101EC00012F0000EF86E390EF76E780EF66EA9EC71
:101ED00012F049EC11F089EC12F040C20EF241C24E
:101EE0000FF242C210F243C211F244C212F245C2D2
:101EF00013F246C214F247C215F248C216F249C2A2
:101F000017F2116A80EC07F0120018C240F219C2F1
:101F100041F21AC242F21BC243F21CC244F21DC279
:101F200045F21EC246F21FC247F220C248F221C249
:101F300049F289EC12F0000EF86E3B0EF76E6A0E55
:101F4000F66EA9EC12F0000EF86E390EF76ED00E98
:101F5000F66EA9EC12F0146A156A166A176A186A06
:101F6000396A3A6AE6DCB8EC12F0FDE3D1EC12F023
:101F70000A0E116201D0E6D00C0E116205D039C0F4
:101F80000AF23AC00BF223D00B0E116201D0116A93
:101F9000300E111216C017F015C016F014C015F04F
:101FA00011C014F0EFEC1EF014C065F015C066F01F
:101FB00016C067F017C068F018C069F01EEC2AF070
:101FC0004FEC22F065C039F066C03AF0CBD789EC0F
:101FD00012F0000EF86E3B0EF76E800EF66EA9EC56
:101FE00012F0000EF86E390EF76ED00EF66EA9ECF8
:101FF00012F0146A156A166A176A186A396A3A6A18
:1020000098DCB8EC12F0FDE3D1EC12F00A0E11628C
:1020100001D098D00C0E116205D039C00CF23AC034
:102020000DF223D00B0E116201D0116A300E111285
:1020300016C017F015C016F014C015F011C014F03A
:10204000EFEC1EF014C065F015C066F016C067F026
:1020500017C068F018C069F01EEC2AF04FEC22F0AF
:1020600065C039F066C03AF0CBD789EC12F0000EAB
:10207000F86E3B0EF76EAC0EF66EA9EC12F019EC92
:102080000DF084C018F285C019F286C01AF287C01C
:102090001BF288C01CF2EEDC84C01DF285C01EF26B
:1020A00086C01FF287C020F288C021F2F0EC0CF04D
:1020B00049EC11F0000EF86E390EF76EBA0EF66E9E
:1020C000A9EC12F0D1EC12F089EC12F0B9EC0BF0A3
:1020D00049EC11F0000EF86E390EF76ED00EF66E68
:1020E000A9EC12F0D1EC12F00A0E116201D02AD044
:1020F0000C0E116227D089EC12F0000EF86E390E2A
:10210000F76E360EF66EA9EC12F0000EF86E390E70
:10211000F76E4C0EF66EA9EC12F005EC11F049ECDE
:1021200011F089EC12F0EEEC0BF049EC11F0000E1E
:10213000F86E390EF76EBA0EF66EA9EC12F0D1EC0D
:1021400012F02AD089EC12F0000EF86E390EF76EFC
:10215000620EF66EA9EC12F0000EF86E390EF76EF4
:10216000780EF66EA9EC12F049EC11F089EC12F041
:1021700040C218F241C219F242C21AF243C21BF223
:1021800044C21CF245C21DF246C21EF247C21FF2F3
:1021900048C220F249C221F280EC07F0116A120015
:1021A000080E956F356A366A396A3A6A4DEC13F053
:1021B000995135269A5136224FEC13F09951392610
:1021C0009A513A22952FF2D7120022EE3BF0050EDB
:1021D000946F140E056E7AEF13F022EE3BF0050EAD
:1021E000946F140E056E82EF13F022EE0EF00A0EBD
:1021F000946F000E056E7AEF13F022EE0EF00A0EC9
:10220000946F000E056E82EF13F022EE18F00A0EA6
:10221000946F0A0E056E7AEF13F022EE18F00A0E94
:10222000946F0A0E056E82EF13F020EE47F0010E58
:10223000946F1C0E056E7AEF13F020EE47F0010E3E
:10224000946F1C0E056E82EF13F020EE45F0010E28
:10225000946F190E056E7AEF13F020EE45F0010E23
:10226000946F190E056E82EF13F020EE51F0010EFF
:10227000946F1A0E056E82EF13F020EE51F0010EEE
:10228000946F1A0E056E7AEF13F049EC11F04BECD7
:1022900011F04BEC11F051EC11F051EC11F051EC4C
:1022A00011F0FA0E11D0C80E0FD0640E0DD0320E00
:1022B0000BD01E0E09D00A0E07D0050E05D0020E57
:1022C00003D0010E01D00D500B6E060E0A6EF80EF3
:1022D000096E092EFED70A2EFCD70B2EF6D7120058
:1022E0000F01806A896A030E386F1F0E926E816A31
:1022F0008A6A000E396F030E936E826A8B6AF00E43
:10230000946E000E3A6F836A8C6A000E956E000E12
:102310003B6F846A8D6A000E3C6F070E966E000E4E
:10232000C16EBE0EC06E000ED06EC00EF16E000EFD
:10233000F06E010E9D6E020EA06EA70ED56E030EFE
:10234000CD6E000EBA6E000EB16E000107D8D00E31
:10235000F26E000ECE6E4C0ECF6E1200946B00EE3D
:1023600000F0EE6A942FFDD7040E956F01EE00F099
:10237000EE6A942FFDD7952FFBD7120080A612008E
:10238000809A8392839057EC11F0200E6AEC12F041
:10239000800E6AEC12F05BEC11F0200E6AEC12F089
:1023A000800E6AEC12F061EC11F0060E5CEC12F09B
:1023B0000C0E5CEC12F0140E5CEC12F02AEC12F035
:1023C000E4EC11F089EF12F089EC12F0000EF86ED7
:1023D0003D0EF76E460EF66EA9EC12F0000EF86E8A
:1023E0003D0EF76E5C0EF66EA9EC12F0000EF86E64
:1023F0003D0EF76E720EF66EA9EC12F0000EF86E3E
:102400003D0EF76E880EF66EA9EC12F049EF11F052
:1024100080A612005F6E74EC12F05F50838283908E
:10242000809AF00B6AEC12F05F38F00B53D05F6EBD
:102430005F465F465F4674EC12F05F5040095CEC0B
:1024400012F0080E946F0900F55008EC12F0942F6A
:10245000FAD7120080A61200000EF86E240EF76E56
:10246000780EF66E080E956F966B965117EC12F07B
:10247000962B952FFAD712000000000000000115DE
:1024800000001010100001150000141414000115B4
:1024900000001515150001150000000000000000E7
:1024A000000000000000000000000000000000002C
:1024B000000000000000000080A612005F6E74ECB7
:1024C00012F05F50F00B83928390809A6AEC12F0C6
:1024D0005F38F00B80A61200E8380F0B826E80A6E2
:1024E0001200808A809A120080A61200828694864A
:1024F000839283809197808A000082A69187809A38
:102500000000808A0000809A91A7F4D79496839067
:102510001200010ED1D7020ECFD7800ECDD7C00E3C
:10252000CBD78009C9D7200E73D780A61200946F2D
:1025300093EC12F0942FFCD7120080A61200606F6B
:10254000603916EC00F008EC12F0605116EC00F067
:102550005FD780A612000900F55091EC12F080A61A
:1025600012000900F55003E008EC12F0FAD712004F
:1025700080A607D0C3EC12F029EC13F002E0D8805B
:1025800001D0D890120080A612008B808B828B84A1
:102590008B86120080A612008B908B928B948B9668
:1025A0001200B8EC12F0FDE3116A03EC13F0116EA7
:1025B000040E946F5BEC11F003EC13F01162F1D791
:1025C000942FF8D7000E11B807D0030E11BA04D01B
:1025D000060E11BC01D0090E956F010E11B404D086
:1025E000020E11B201D0030E952795C011F0640EB2
:1025F000946FB8EC12F006E35BEC11F0942FF9D76E
:10260000100E1126120080A61200CAEC12F08B8068
:1026100029EC13F015E1CAEC12F08B8229EC13F0CF
:102620000FE1CAEC12F08B8429EC13F009E1CAEC3B
:1026300012F08B8629EC13F003E1956BE86A120027
:102640008250E838F00B956F29EC13F09511CAEF22
:1026500012F080A612008450070BE8A002D0040EEE
:1026600002D0E8B4010E120080A61200116AB8EC84
:1026700012F0FAE3120080A61200B8EC12F0FBE2AE
:1026800012001D0E0DD0190E0BD0150E09D0110E13
:1026900007D00D0E05D0090E03D0050E01D0010E96
:1026A000C26E17EC08F0C282C2B2FED7C4CF9AF055
:1026B000C3CF99F01200A6B2FED705C0A9FF06C08D
:1026C000A8FFA69EA69CA684F29EF2BEFDD7550E3C
:1026D000A76EAA0EA76EA68207A0F28EA69412007D
:1026E000A6B2FED705C0A9FFA69EA69CA680A8CF2D
:1026F00006F01200DECF06F05BEC13F0052A942FF3
:10270000F9D7120070EC13F006C0DEFF052A942FF3
:10271000F9D71200000EF86E370EF76ED40EF66E73
:10272000A9EC12F0FDEC1EF096C06FF051EC29F010
:10273000020E8E6F8F6B5CEC28F0010E966308D052
:10274000000EF86E3B0EF76EE60EF66EA9EC12F078
:10275000020E966308D0000EF86E3B0EF76EFC0E6C
:10276000F66EA9EC12F0030E966308D0000EF86E18
:102770003C0EF76E120EF66EA9EC12F0040E966384
:1027800008D0000EF86E3C0EF76E280EF66EA9EC1F
:1027900012F0050E966308D0000EF86E3C0EF76E30
:1027A0003E0EF66EA9EC12F0060E966308D0000EEF
:1027B000F86E3C0EF76E540EF66EA9EC12F0070E92
:1027C000966308D0000EF86E3C0EF76E6A0EF66E39
:1027D000A9EC12F0080E966308D0000EF86E3C0EBD
:1027E000F76E800EF66EA9EC12F0090E966308D013
:1027F000000EF86E3C0EF76E960EF66EA9EC12F017
:102800000A0E966308D0000EF86E3C0EF76EAC0E02
:10281000F66EA9EC12F00B0E966308D0000EF86E5F
:102820003C0EF76EC20EF66EA9EC12F00C0E96631B
:1028300008D0000EF86E3C0EF76ED80EF66EA9ECBE
:1028400012F00D0E966308D0000EF86E3C0EF76E77
:10285000EE0EF66EA9EC12F00E0E966308D0000E86
:10286000F86E3D0EF76E040EF66EA9EC12F00F0E28
:10287000966308D0000EF86E3D0EF76E1A0EF66ED7
:10288000A9EC12F0100E966308D0000EF86E3D0E03
:10289000F76E300EF66EA9EC12F0120080A6120050
:1028A00089EC12F0000EF86E370EF76EA80EF66E79
:1028B000A9EC12F0000EF86E370EF76EBE0EF66E33
:1028C000A9EC12F0010E966FB5EC07F0800E346E95
:1028D000080E966504D034C033F0326A03D034C099
:1028E00032F0336AFCEC07F015DFD1EC12F0030E86
:1028F000116212D0962B090E966303D0800E346EAF
:10290000E7D7110E966305D0010E966F800E346ED8
:10291000DFD7D8903432DCD7010E116211D0960780
:10292000080E966303D0010E346ED2D7966705D099
:10293000100E966F010E346ECBD7D8903436C8D7B0
:1029400089EC12F0FF0083885BEC11F08398120091
:1029500055EC11F002D855EC11F0838855EC11F0CC
:102960008398120083941AD817D8838406D819D074
:10297000838414D811D8839406D88396000000006D
:102980000000000000000000000000000000000047
:1029900000000000000012008386F0D79594959601
:1029A0001200958495861200E3DFA00E0BD858BE66
:1029B000FBD75A5007D858BEF7D7595003D858BE3E
:1029C000F3D7120083965D6EE9DF080E5E6E838496
:1029D0005DAE8394D8DFE0DFD0DF5D365E2EF7D7C3
:1029E00095849596589ED8DF83B4588ECCDF839615
:1029F0001200080E5E6E5B6A5B365B90F1DF58BEBC
:102A00005B805E2EF9D71200CFDF5C50DBDFAAD7E8
:102A1000A9DFCADFADDFA10ED5DF58BEF9D7E9DFE8
:102A2000A1D7766703D0776701D01BD06FC059F06C
:102A300070C05AF009EC15F05BC05CF074C059F03E
:102A400075C05AF004EC15F06F2BD8B4702B742BB2
:102A5000D8B4752B76077629D8B47707D8B47653CF
:102A6000E0D7120009EC15F05BC06FF0592AD8B41A
:102A70005A2A09EC15F05BC070F0592AD8B45A2ACA
:102A800009EC15F05BC071F0592AD8B45A2A09EC48
:102A900015F05BC072F0E8686F5D18E0060E6F61BC
:102AA00015D0830E746F030E756F7251755D02E160
:102AB0007151745DD8A00AD06FC01CF070C01DF0B9
:102AC00071C01EF072C01FF0D89001D0D8801200E3
:102AD0001CC05CF004EC15F0592AD8B45A2A1DC069
:102AE0005CF004EC15F0592AD8B45A2A1EC05CF0E8
:102AF00004EC15F0592AD8B45A2A1FC05CF004EC33
:102B000015F01200EFEC1EF07AC16FF07BC170F08F
:102B1000B80E746F0B0E756F7051755D02E16F51D9
:102B2000745DD8A00CD0960E746F000E756F705146
:102B3000755D02E16F51745DD8B001D002D0D890BC
:102B40003AD0960E746F000E756F70EC22F0F7ECB1
:102B50001FF004EC1FF0040E746FF1EC26F0010E70
:102B6000456204D0000E746F000E756F020E456250
:102B700004D0880E746F2C0E756F030E456204D05E
:102B8000100E746F590E756F040E456204D0980EC6
:102B9000746F850E756F050E456204D0200E746F3C
:102BA000B20E756F74516F27755170236FC059F055
:102BB00070C05AF0D88012006F6B706B010E1A62F1
:102BC00005D0000E6F6F000E706F1FD0020E1A62DC
:102BD00005D0880E6F6F2C0E706F17D0030E1A621F
:102BE00005D0100E6F6F590E706F0FD0040E1A6261
:102BF00005D0980E6F6F850E706F07D0050E1A62A4
:102C000004D0200E6F6FB20E706F120089EC12F0BC
:102C1000000EF86E3A0EF76E200EF66EA9EC12F06A
:102C2000000EF86E3A0EF76E4C0EF66EA9EC12F02E
:102C30008388C2DF880E746F2C0E756F6FC059F0D9
:102C400070C05AF0756703D0746701D00ED0FF0EC4
:102C50005C6E04EC15F0592AD8B45A2A740774290A
:102C6000D8B47507D8B47453EDD7839889EC12F0B3
:102C7000000EF86E3A0EF76E0A0EF66EA9EC12F020
:102C800055EC11F0120089EC12F0000EF86E3A0EBD
:102C9000F76E360EF66EA9EC12F0000EF86E3A0ED4
:102CA000F76E4C0EF66EA9EC12F08388060E1660D5
:102CB0001AD0060E176017D01750165CD8B413D070
:102CC0000C0E186210D017C01AF076DF6FC074F0C7
:102CD00070C075F016C01AF06FDF880E766F2C0E7C
:102CE000776F11EC15F0C1D783887AC190F17BC161
:102CF00091F17AC16FF07BC170F06F6703D070679C
:102D000001D0D1D089EC12F0000EF86E3A0EF76EB9
:102D1000140EF66EA9EC12F04BEC11F0C80E4A6ED0
:102D2000000E4B6E70514B5C02E16F514A5CD8A0B3
:102D300005D0B40E486E000E496E90D0860E4A6ED5
:102D4000010E4B6E70514B5C02E16F514A5CD8A092
:102D500005D0540E486E010E496E80D01A0E4A6E90
:102D6000020E4B6E70514B5C02E16F514A5CD8A071
:102D700005D0160E486E020E496E70D0DA0E4A6EFD
:102D8000020E4B6E70514B5C02E16F514A5CD8A051
:102D900005D0B20E486E020E496E60D0010E4A6E2A
:102DA000040E4B6E70514B5C02E16F514A5CD8A02F
:102DB00005D0E80E486E030E496E50D0A00E4A6E44
:102DC000050E4B6E70514B5C02E16F514A5CD8A00E
:102DD00005D06E0E486E050E496E40D01C0E4A6E30
:102DE000070E4B6E70514B5C02E16F514A5CD8A0EC
:102DF00005D0080E486E070E496E30D0700E4A6E30
:102E0000080E4B6E70514B5C02E16F514A5CD8A0CA
:102E100005D02A0E486E080E496E20D0C40E4A6EA8
:102E2000090E4B6E70514B5C02E16F514A5CD8A0A9
:102E300005D0920E486E090E496E10D0B80E4A6E3B
:102E40000B0E4B6E70514B5C02E16F514A5CD8A087
:102E500005D0E60E486E0A0E496E00D048C07AF1E1
:102E600049C07BF182EC15F068EC15F04B50495CE1
:102E700002E14A50485CD8B404D0482AD8B4492A60
:102E8000EDD789EC12F0000EF86E3A0EF76E0A0ECE
:102E9000F66EA9EC12F0A8EC14F04BEC11F089ECF2
:102EA00012F0D89015D0000EF86E390EF76EE60EBF
:102EB000F66EA9EC12F0000EF86E390EF76EF80EF1
:102EC000F66EA9EC12F04BEC11F089EC12F0D88000
:102ED00090C17AF191C17BF18398120083887AC105
:102EE00090F17BC191F17AC148F07BC149F07AC180
:102EF0004AF07BC14BF01A50485E1B50495A1A5099
:102F00004A261B504B22AAD7000EF86E390EF76ED8
:102F1000E60EF66EA9EC12F0000EF86E390EF76EA2
:102F2000F80EF66EA9EC12F04BEC11F089EC12F0F1
:102F3000D88012008388056A946B24EE00F082EC3E
:102F400013F0000E596EDF0E5A6E24EE00F0946BF3
:102F5000DECF5CF004EC15F0592AD8B45A2A942F2D
:102F6000F7D745EC11F0839812008388000E596E54
:102F7000DF0E5A6E24EE00F0946B09EC15F05BC086
:102F8000DEFF592AD8B45A2A942FF7D700C46FF01D
:102F90006F2909E0056A946B24EE00F07AEC13F0D7
:102FA00045EC11F0FF008398120000526561646DDA
:102FB000656D6F72792020202020202020202000A5
:102FC00000526561646D656D6F727920545255458C
:102FD00020202020200000526561646D656D6F72B5
:102FE000792046414C5345202020200082EC15F0EA
:102FF00009E332EC15F006E2078A640E426ED890BF
:1030000095EF07F0D88012003D92010E1A6208D0A9
:10301000540E2E6E0A0E2F6E230E306E080E316E79
:10302000020E1A6208D0230E2E6E080E2F6EE90EC5
:10303000306E060E316E030E1A6208D0E90E2E6E47
:10304000060E2F6E140E306E060E316E040E1A62CE
:1030500008D0140E2E6E060E2F6E760E306E050EF4
:10306000316E050E1A6208D0760E2E6E050E2F6E8A
:10307000FA0E306E040E316E060E1A6208D0FA0E89
:103080002E6E040E2F6E950E306E040E316E070EEE
:103090001A6208D0950E2E6E040E2F6E400E306E02
:1030A000040E316E080E1A6208D0400E2E6E040E09
:1030B0002F6EF80E306E030E316E090E1A6208D0B4
:1030C000F80E2E6E030E2F6EBA0E306E030E316E9A
:1030D0001A6601D003D0080E4E6E07D03D82E90E6D
:1030E000306E060E316E080E4E6E079889EC12F0A7
:1030F000000EF86E3A0EF76EC60EF66EA9EC12F0E0
:10310000000EF86E3A0EF76EDC0EF66EA9EC12F0B9
:1031100007B8C1D05DEC05F0FBE389EC12F0000EBE
:10312000F86E3A0EF76EC60EF66EA9EC12F0A6EC2B
:1031300002F083884BEC11F0839889EC12F0010EB9
:10314000226E22C021F0EFEC1EF01EC06FF01FC0F7
:1031500070F0640E746F65EC27F06F5106E1236A1E
:10316000246A630E256E000E266E010E656308D07C
:10317000640E236E000E246EC70E256E000E266EA2
:10318000020E656308D0C80E236E000E246E2B0E4F
:10319000256E010E266E030E656308D02C0E236E7D
:1031A000010E246E8F0E256E010E266E040E6563D1
:1031B00008D0900E236E010E246EF30E256E010EC4
:1031C000266E050E656308D0F40E236E010E246E84
:1031D000570E256E020E266E060E656308D0580E39
:1031E000236E020E246EBB0E256E020E266E070E97
:1031F000656308D0BC0E236E020E246E1F0E256E72
:10320000030E266E080E656308D0200E236E030E93
:10321000246E830E256E030E266E206A1BEC1AF0B8
:103220002BC01DF02CC01EF02DC01FF0B9EC07F014
:1032300033EC1BF089EC12F0000EF86E3A0EF76ECC
:10324000C60EF66EA9EC12F03DA015D0000EF86E79
:103250003A0EF76EE80EF66EA9EC12F0000EF86E5C
:103260003A0EF76EF40EF66EA9EC12F0E00E406E18
:103270002E0E416E10D0000EF86E3A0EF76EE80E6C
:10328000F66EA9EC12F0000EF86E3A0EF76EFC0E18
:10329000F66EA9EC12F057EC19F089EC12F00798D1
:1032A0003DA004D01A6A1B6A6EEC17F012008378F6
:1032B0003DA055EC11F03DB04BEC11F034EC00F0BA
:1032C000F6E28398120059EF11F0FDDFD0EC10F018
:1032D00035C054F036C055F0200E6F6F030E706F7E
:1032E0006F515426705155223950545E3A50555AF8
:1032F00055AE02D0546A556A12001C6603D01E6A8D
:103300001F6A18D0746B756B22C074F074511E263E
:1033100075511F2225C074F026C075F01F50755DD1
:1033200002E11E50745DD8B005D0078625C01EF09E
:1033300026C01FF012001C6603D01E6A1F6A1DD033
:10334000746B756B22C074F074511E5E75511F5AF8
:103350001FAE08D00786BDEC1AF023C01EF024C0B3
:103360001FF00BD023C074F024C075F01F50755DA2
:1033700002E11E50745DD8B0EDD71200050E1C623C
:1033800002D01D6A12D0746B756B766B776B21C09F
:1033900074F01DC076F0745176277551772376C08E
:1033A0001DF0775302E007861D681200050E1C62AF
:1033B00002D01D6A14D0746B756B766B776B21C06D
:1033C00074F01DC076F07451765F7551775B76C0EE
:1033D0001DF077AF04D00786BDEC1AF01D6A12000D
:1033E000205202E1A8DF26D0010E206203D0A3DF25
:1033F000DDDF20D0020E206202D0D8DF1BD0030E0A
:10340000206203D0D3DF79DF15D0040E206202D012
:1034100074DF10D0050E206203D06FDFAFDF0AD05B
:10342000060E206202D0AADF05D0070E206202D06D
:10343000A5DF81DF12003D9065EC19F054C027F044
:1034400055C028F01DC02BF01EC02CF01FC02DF061
:103450004EC04DF00A0E4C6E526A536A4F6A522AA1
:1034600007B875D065EC19F05550285C02E154504E
:10347000275CD8B00DD01DC02BF01EC02CF01FC093
:103480002DF054C027F055C028F052C053F04F2AF9
:10349000F0EC19F0B9EC07F04C2EE1D789EC12F002
:1034A0002BC01DF02CC01EF02DC01FF0B9EC07F092
:1034B00065EC19F00EEC02F0BFEC00F022C26FF0E8
:1034C00023C270F024C271F025C272F026C273F0DC
:1034D00073AF02D007883BD0F6EC00F02DEC01F082
:1034E00075EC01F0A2EC01F03DB20FD02EC06FF0F0
:1034F0002FC070F08AC174F08BC175F07051755D8A
:1035000002E16F51745DD8B021D053520DE04EC02E
:103510004DF0020E4F6009D0030E536002D020D848
:1035200004D0090E536001D023D84D2E93D730C05C
:103530006FF031C070F08AC174F08BC175F07551B5
:10354000705D02E174516F5DD8B001D03D80120012
:10355000040E2026070E206402D0080E205E0DD037
:10356000020E2026070E206402D0080E205E05D031
:10357000202A080E206201D0206A4CD80EE3206673
:1035800002D0020E206E010E206202D0020E206ECA
:10359000070E206202D0060E206E31D80FE3030E14
:1035A000206202D0020E206E040E206202D0020EB3
:1035B000206E050E206202D0060E206E1D660ED013
:1035C000020E206202D0040E206E030E206202D092
:1035D000040E206E010E206201D0206A1D280EE12B
:1035E000050E206202D0040E206E060E206202D06C
:1035F000040E206E070E206201D0206A12001F50B8
:10360000265C02E11E50255CD8A402D0D8801200AE
:10361000D89012001F50245C02E11E50235CD8A4F5
:1036200002D0D8801200D89012008C928C908B9689
:103630008B948B92120080B61200F7DF010E456268
:1036400001D08C82020E456201D08C80030E45624F
:1036500001D08B86040E456201D08B84050E456235
:1036600001D08B8212004FEC11F0D0EC10F035C07D
:1036700037F036C038F0BFEC00F088EC00F0F6EC24
:1036800000F02DEC01F04BEC00F03BC08EF13CC0A3
:103690008FF13BC08CF13CC08DF11200EACF04F0F9
:1036A000E9CF03F0F2A401D0F294F2A203D0078292
:1036B0000788F2929EA013D09E904266420643660F
:1036C0004306415202E1405206E040064028D8B489
:1036D0004106D8B44052000ECE6E4C0ECF6EA1B84B
:1036E000A1989EA201D09E9204C0EAFF03C0E9FF08
:1036F0001100006ED8CF01F0E0CF02F002C0E0FF71
:10370000005001C0D8FF1000000EF86E370EF76EA3
:10371000500EF66EA9EC12F01200000EF86E370E85
:10372000F76E660EF66EA9EC12F01200000EF86E3F
:10373000370EF76E7C0EF66EA9EC12F01200000E3A
:10374000F86E370EF76E920EF66EA9EC12F01200BC
:103750000020202020202020202020202020202089
:103760002020202020004020202020202020202059
:103770002020202020202020202020001420202075
:103780002020202020202020202020202020202039
:103790002000542020202020202020202020202015
:1037A000202020202020200000203D3D3D2052658B
:1037B0006C61697374657374203D3D3D2000543322
:1037C0002D566F7220312D5A75727565636B2023EB
:1037D0002D3E5800402050494E3A2058312D41008E
:1037E00000203D3D20536368726974746D6F746F7F
:1037F00072203D3D200040202D2D204461756572D2
:1038000074657374202D2D2D2D2D200014416262BE
:10381000727563682D3E2054617374652C44544D59
:10382000460014202D2D20416262727563682121AB
:10383000202D2D2D2D2D200040204E756C6C706F8D
:10384000736974696F6E2073756368656E004020DC
:10385000506F736974696F6E20676566756E646515
:103860006E2021004020506F732E6E6963687420B3
:10387000676566756E64656E210000433A00404CD2
:103880003A0014503A00544600000D563A004C528B
:103890004C3A00001F5357523A00062D4C2D0000A1
:1038A000462020200000062D4C2B000046202043FF
:1038B0000000062B4C2D0000464320200000062D62
:1038C000432B00004620204C0000062B432D000017
:1038D000464C20200000062D432D000046202020CD
:1038E00000000A4100004D487A0000566F726C617A
:1038F000756620202020202020202020202020004D
:1039000000527565636B6C61756620202020202055
:103910002020202020004020203064426D3A00000A
:10392000402D333064426D3A0000006B783A00005D
:10393000406B793A0000004B616C69627269657294
:10394000756E6720204F4B2020202000406D6B7843
:103950002C206D6B792073706569636865726E20C9
:103960002000004B616C696272696572756E672038
:103970004162627275636800406D6B782C206D6BDC
:103980007920726573746F72652020202000545373
:1039900070656963682E39202041626272756368C0
:1039A000202320005457656974657220332020411C
:1039B00062627275636820232000545461737465D9
:1039C000202D3E205765697465722020202020003C
:1039D00054576569746572202320204162627275B4
:1039E0006368202A2000004B65696E652046726579
:1039F0007175656E7A2D200040696E666F726D611B
:103A000074696F6E20212120200000466572746960
:103A10006721210000536176652042616E642100B8
:103A2000003D20416E74656E6E65206C6F6573633A
:103A300068656E203D00003D20416E74656E6E65C8
:103A4000206B6F70696572656E203D004057617232
:103A500074656E2021212100003D205345545550AE
:103A6000203D202023204162627275636800404D32
:103A70004B766F7220205B315D4B616C5B335D5622
:103A800069657700144D4B727565636B5B325D4BF6
:103A9000616C5B345D5669657700404B616C2E76D6
:103AA0006F72206D616E75656C6C20205B315D00FE
:103AB000144B616C2E727565636B206D616E75655C
:103AC0006C6C5B325D00003D3D3D3D204E616368A6
:103AD00074756E656E20203D3D3D3D00145761724A
:103AE00074656E20545821004041627374696D6D95
:103AF000756E6700144F4B2021210000146E69631E
:103B000068747320676566756E64656E2100004198
:103B1000444355766F7220203A0000414443557269
:103B20007565636B3A0000414443766F7220203A1A
:103B3000000000414443727565636B3A0000145005
:103B40006567656C313A203064426D20202020206A
:103B50002020200014506567656C323A202D3330E8
:103B600064426D202020202020001445696E67618A
:103B70006265203064426D2020202020202020001B
:103B80001445696E67616265202D333064426D2093
:103B9000202020202000003D3D2041443833303794
:103BA00020566F726C617566203D3D00003D2041DE
:103BB000443833303720527565636B6C617566200D
:103BC0003D00406D6B783A00146D6B793A004041CE
:103BD000444320203064426D3A00144144432D3365
:103BE0003064426D3A00146C5F676C312C4B312CA1
:103BF000322020202020203136754800146C5F6769
:103C00006C312C4B332C3420202020202020387580
:103C10004800146C5F676C312C4B352C362020200B
:103C20002020202034754800146C5F676C312C4BC9
:103C3000372C382020202020202032754800146C9A
:103C40005F676C322C4B392C313020202020202013
:103C500031754800146C5F676C322C4B31312C315C
:103C6000322020203530306E4800146C5F676C3293
:103C70002C4B31332C31342020203235306E48002B
:103C8000146C5F676C322C4B312C322020202020AA
:103C90003132356E480014635F676C6965642C20AF
:103CA00052656C616973204B3320200014635F6799
:103CB0006C6965642C2052656C616973204B3220FD
:103CC000200014635F676C6965642C2052656C6129
:103CD0006973204B3120200014635F676C69656451
:103CE0002C2052656C616973204B34202000146CC9
:103CF0005F676C696564322C2052656C6169732062
:103D00004B342000146C5F676C696564322C205260
:103D1000656C616973204B332000146C5F676C69BC
:103D20006564312C2052656C616973204B39200029
:103D3000146C5F676C696564312C2052656C616935
:103D400073204B31300000202053796D54756E651F
:103D5000722037353057617474202000403D3D3D5E
:103D60003D3D3D3D3D3D3D3D3D3D3D3D3D3D3D3D83
:103D70003D00142D204857312E303120286329442E
:103D80004C344A414C202D00542D205357322E30B4
:103D900034202032392E31312E3139202D002D2D75
:103DA0002D00494E46006D570000755700006E57B4
:103DB0000000705700006657000061570000572050
:103DC00000006B570000205600006D56000075562D
:103DD00000006E56000064426D007373000013D83B
:103DE00006D86A6B6B6B6C6B6D6B6E6B1200656BE0
:103DF000666B676B686B696B12006F6B706B716BD6
:103E0000726B736B1200F9DF746B756B766B776B8B
:103E1000786B1200846B856B866B876B886B1200E6
:103E20000EC189F00FC18AF010C18BF011C18CF066
:103E300012C18DF012000EC184F00FC185F010C1C7
:103E400086F011C187F012C188F0120089C084F099
:103E50008AC085F08BC086F08CC087F08DC088F05A
:103E6000120084C089F085C08AF086C08BF087C0BC
:103E70008CF088C08DF0120084C00EF185C00FF167
:103E800086C010F187C011F188C012F1120013C171
:103E900084F014C185F015C186F016C187F017C1F2
:103EA00088F0120013C189F014C18AF015C18BF09B
:103EB00016C18CF017C18DF0120018C184F019C121
:103EC00085F01AC186F01BC187F01CC188F0120072
:103ED00018C189F019C18AF01AC18BF01BC18CF08E
:103EE0001CC18DF012001DC184F01EC185F01FC1E0
:103EF00086F020C187F021C188F012001DC189F031
:103F00001EC18AF01FC18BF020C18CF021C18DF041
:103F1000120022C184F023C185F024C186F025C19E
:103F200087F026C188F0120022C189F023C18AF0EF
:103F300024C18BF025C18CF026C18DF0120027C161
:103F400084F028C185F029C186F02AC187F02BC1F1
:103F500088F0120027C189F028C18AF029C18BF0AE
:103F60002AC18CF02BC18DF0120089C013F18AC0D8
:103F700014F18BC015F18CC016F18DC017F1120031
:103F800084C013F185C014F186C015F187C016F105
:103F900088C017F1120084C018F185C019F186C0DD
:103FA0001AF187C01BF188C01CF1120084C01DF1FA
:103FB00085C01EF186C01FF187C020F188C021F1A5
:103FC000120084C022F185C023F186C024F187C08D
:103FD00025F188C026F1120084C027F185C028F1A0
:103FE00086C029F187C02AF188C02BF1120065C074
:103FF0006FF066C070F067C071F068C072F069C0A1
:1040000073F0120065C074F066C075F067C076F09A
:1040100068C077F069C078F012006FC065F070C0BA
:1040200066F071C067F072C068F073C069F012008A
:104030007437753776377737783712006F377037C0
:1040400071377237733712007833773376337533BD
:104050007433120073337233713370336F33120061
:1040600006D86A376B376C376D376E371200653795
:10407000663767376837693712006E336D336C33D4
:104080006B336A331200F9DF6933683367336633A1
:10409000653312006FAF04D070697169726973691A
:1040A000120070AF03D0716972697369120071AF49
:1040B00002D072697369120072AF01D07369120085
:1040C000929391BF92838CDE280E626FD8902AEC77
:1040D00020F044EC20F003D8622FF8D7120033EC24
:1040E0002AF00A0E616F00EE65F0EF50E8B6FD0FA2
:1040F000E8BED00FEE6E612FF8D740EC2AF0120028
:104100003FD869AF09D06A2BD8B46B2BD8B46C2BCD
:10411000D8B46D2BD8B46E2BF7EC1EF035D030D858
:1041200069AF09D06A2BD8B46B2BD8B46C2BD8B438
:104130006D2BD8B46E2B6AC065F06BC066F06CC096
:1041400067F06DC068F06EC069F091BF38EC27F081
:10415000120016D86AC065F06BC066F06CC067F0DC
:104160006DC068F06EC069F091BF38EC27F01200A6
:1041700007D8F1EC1EF008D003D8F7EC1EF004D0FD
:10418000D3EC22F0C8EF20F085EC21F0E9EF22F02B
:104190004CD803E1F0EC1EF01AD01AD87F0E796FDC
:1041A00079517D5F7A517E5B7DC061F07D530FE078
:1041B0007DBF06D0D89030EC20F0612FFBD707D020
:1041C000611F612BD89043EC20F0612FFBD71200C8
:1041D000919F83BF918F839FF0EC1EF07FC066F0AC
:1041E00080C067F081C068F082C069F083C06AF067
:1041F000D89030EC20F044EC20F0698F6AC07DF05C
:104200006A6BD89030EC20F01200040E616FEE66FD
:1042100008D0612FFCD7EECFE8FF7F0B03E1D884F5
:1042200001D0D89440EC2AF0120033EC2AF000EED2
:104230007FF0EBD733EC2AF000EE84F0E6D733ECD6
:104240002AF000EE89F0E1D733EC2AF000EE6FF0AF
:10425000DCD733EC2AF000EE74F0D7D733EC2AF039
:1042600000EE65F00A0E616FEE66DBD7612FFCD7BA
:10427000D6D7736B72BF736935D0726B736B71AFC6
:1042800031D0726973692ED0716B726B736B70AFC2
:1042900029D071697269736925D0706B716B726B0B
:1042A000736B6FAF1FD070697169726973691AD0CF
:1042B000F0EC1EF0919F736B1DD0F0EC1EF0919FFF
:1042C000726B736B17D0F0EC1EF0919F716B726B79
:1042D000736B10D0F0EC1EF0919F706B716B726B72
:1042E000736B08D0F0EC1EF0919F73AF03D047ECD6
:1042F00027F0918F6FC06AF070C06BF071C06CF0E6
:1043000072C06DF073C06EF000D07F0E7D6F000E36
:104310007E6F2EEC21F006E17F6B806B816B826BF0
:10432000836B36D0EFEC21F007E0D89043EC20F01F
:104330007D2BD8B47E2BF6D76AB10AD0D89030EC5A
:1043400020F07D077D29D8B47E07D8B47D53F4D7FB
:1043500066A10BD06681662BD8B4672BD8B4682BC6
:10436000D8B4692BD8B46A2BDDD7656B6A917DC050
:104370006AF043EC20F066C07FF067C080F068C050
:1043800081F069C082F06AC083F0839F91BF838F00
:1043900012007F6B806B816B836B800E826FF5D711
:1043A0007F69806981697F0E826F7F0E836FEDD791
:1043B0007F0E6F6F000E706F7E51705D02E17D5158
:1043C0006F5DD8B003D0ECDFD88401D0D894120050
:1043D0007EAF03D0DEDFD88401D0D894120033EC56
:1043E0002AF000EE6EF0040E616FED660AD0612FC8
:1043F000FCD7010EEF6201D002D0EF6602D0D88464
:1044000001D0D89440EC2AF0120074C000F175C0BD
:1044100001F176C002F177C003F178C004F14FECEE
:1044200022F065C007F166C008F167C009F168C0F5
:104430000AF169C00BF100C16FF001C170F002C157
:1044400071F003C172F004C173F035EC22F007C1C2
:104450006AF008C16BF009C16CF00AC16DF00BC1C4
:104460006EF0919F92B3918F1200BADC280E626FAA
:10447000D89005D837EC20F0622FFAD7120033EC31
:104480002AF0050E616F00EE6FF0D890EF50E82033
:104490000700EE6E612FFAD740EC2AF0120033ECE1
:1044A0002AF09EDC280E626FD8902AEC20F044ECB3
:1044B00020F000EE6FF0050E616FEFAE02D0300E0F
:1044C000EF5EEFA602D0030EEF5EEE52612FF5D73E
:1044D000622FEAD740EC2AF0120002D8F7EF1FF063
:1044E00033EC2AF09ADD00EE65F010EE74F0040E65
:1044F000616FE650EE5EE650EE5A612FFCD740EC5D
:104500002AF0120002D8F7EF1FF033EC2AF085DD15
:1045100000EE65F010EE74F0E650EE26040E616FCA
:10452000E650EE22612FFCD740EC2AF0120000C1C9
:104530006FF001C170F002C171F003C172F004C1EB
:1045400073F005C179F006C17AF0120007C174F06A
:1045500008C175F009C176F00AC177F00BC178F097
:104560000CC17BF00DC17CF0120066C000F167C089
:1045700001F168C002F169C003F16AC004F17DC0B5
:1045800005F17EC006F1120066C007F167C008F1B0
:1045900068C009F169C00AF16AC00BF17DC00CF175
:1045A0007EC00DF1120084C07FF085C080F086C00F
:1045B00081F087C082F088C083F0120089C07FF04C
:1045C0008AC080F08BC081F08CC082F08DC083F0F7
:1045D00012007FC084F080C085F081C086F082C068
:1045E00087F083C088F012007FC089F080C08AF015
:1045F00081C08BF082C08CF083C08DF0120050EC33
:104600002AF016E24DEC2AF013E21AEC21F01AE03F
:104610001FEC21F017E065EC2AF004E31AEC21F01E
:1046200001E306D068EC2AF006E31FEC21F003E377
:104630008DEC2AF0120065EC2AF003E382EC2AF0FC
:1046400003D00DD00AEC1FF088BF03D08DAF01D08E
:10465000888F88AF03D08DBF01D0888F12001DD8FE
:10466000919F91BB917F91BD917FF4EC26F069C041
:1046700000F16AC001F16BC002F16CC003F16DC0C2
:1046800004F11ED885EC22F0F7EC1FF004EC1FF0CB
:104690007F0E746F70EC22F01ED0919B919D88BFAD
:1046A000918B8DBF918D7FDFE8EC20F05EDF86DFA0
:1046B000E8EC20F069DFEFEC1EF039DFA6EF22F026
:1046C000EFEC1EF079C06FF07AC070F07BC074F030
:1046D0007CC075F0120065C07DF066C07EF0F0EC25
:1046E0001EF000C166F001C167F002C168F003C1AD
:1046F00069F004C16AF089EC21F0E9EF22F050EC96
:104700002AF009E24DEC2AF006E21AEC21F006E16B
:104710001FEC21F019E18DEC2AF0120068EC2AF070
:1047200003E365EC2AF0F7E21FEC21F010E182ECE4
:104730002AF088BF03D08DAF01D0888F88AF03D017
:104740008DBF01D0888F120097EC2AF0F2D7A5DF39
:10475000919F91BB917F91BD917FC2EC27F005DFC6
:10476000AFDF70EC22F0F7EC1FF004EC1FF07F0ECF
:10477000746F85EC22F0AFD71FEC21F001E112003D
:104780008D7F00D050EC2AF004E24DEC2AF001E2DB
:1047900003D08DEC2AF012001FEC21F001E1120091
:1047A0001AEC21F003E126EC1FF0120017D885EC7B
:1047B00022F079C07DF07AC07EF0919F69AF03D07E
:1047C000918F38EC27F065C000F166C001F167C039
:1047D00002F168C003F169C004F181D75EDFFE0E0B
:1047E0007D6F000E7E6F7C517A5D02E17B51795DB9
:1047F00027E013E37B2BD8B47C2B7E517C5D02E158
:104800007D517B5D07E104EC1FF079C07BF07AC03D
:104810007CF016D0D89018DCE6D7792BD8B47A2B58
:104820007E517A5D02E17D51795D07E1FDEC1EF07C
:104830007BC079F07CC07AF003D0D8900BDCD3D762
:1048400091BB47EC27F091BD56EC27F0120031ECFC
:104850001FF0FFEF22F01AEC21F02DE088BF2CD0E2
:1048600050EC2AF028E23CEC1FF0ECD848DFC0EC1A
:104870001FF01E0E646F644F1ED01BEC1FF052EC35
:104880001FF03DDF52EC1FF07DDFDCD838DF52EC4B
:104890001FF08D51885D0BE18C51875D08E18B51D4
:1048A000865D05E18A51855D02E18951845D03E001
:1048B000C0EC1FF0E0D712008DEC2AF012001AECC9
:1048C00021F008E13F0E886F800E876F846B856B47
:1048D000866B120001013F0E266F800E256F226B42
:1048E000236B246B3F0E216F800E206F1D6B1E6BA0
:1048F0001F6B0001CBEC1FF0C0EC1FF022C10EF1CA
:1049000023C10FF124C110F125C111F126C112F10B
:104910001E0E646F47EC1FF07EEC1FF0F0DE10EC13
:104920001FF0C2EC23F010EC1FF08D51885D0BE1FD
:104930008C51875D08E18B51865D05E18A51855D6B
:1049400002E18951845D17E0644F15D03CEC1FF003
:1049500089EC1FF06FD816DFE1EC1FF07EEC1FF042
:104960004EDED6EC1FF05DEC1FF052EC1FF047DE80
:10497000C0EC1FF0CFD712001AEC21F008E13F0E77
:10498000886F800E876F846B856B866B120084C086
:104990002CF185C02DF186C02EF187C02FF188C083
:1049A00030F1B8EC20F03BD82ADE89DFECEC1FF0C8
:1049B0002CC184F02DC185F02EC186F02FC187F067
:1049C00030C188F0C0EC20F0919591BF91856AC00C
:1049D00064F027C184F028C185F029C186F02AC17E
:1049E00087F02BC188F0645306E091A5C5D891B536
:1049F000D5D8642FFAD71200420E8D6F480E8C6FF7
:104A0000896B8A6B8B6B1200400E8D6F490E8C6F19
:104A10000F0E8B6FDA0E8A6FA20E896F1200400E96
:104A20008D6F130E8C6F5D0E8B6F8D0E8A6FDE0E89
:104A3000896F12003F0E8D6F800E8C6F896B8A6BB1
:104A40008B6B1200400E8D6F896B8A6B8B6B8C6B3E
:104A50001200410E8D6F200E8C6F896B8A6B8B6BF1
:104A60001200420E8D6FC80E8C6F896B8A6B8B6B38
:104A70001200440E8D6F7A0E8C6F896B8A6B8B6B74
:104A80001200460E8D6F1C0E8C6F400E8B6F896B63
:104A90008A6B1200470E8D6FC30E8C6F500E8B6F9A
:104AA000896B8A6B1200490E8D6F740E8C6F240E09
:104AB0008B6F896B8A6B12004B0E8D6F180E8C6F8B
:104AC000960E8B6F800E8A6F896B12004C0E8D6F65
:104AD000BE0E8C6FBC0E8B6F200E8A6F896B12001E
:104AE0004E0E8D6F6E0E8C6F6B0E8B6F280E8A6F55
:104AF000896B12003D0E8D6FCC0E8C6FCC0E8B6FC0
:104B0000CC0E8A6FCD0E896F12003C0E8D6F230E76
:104B10008C6FD70E8B6F0A0E8A6F3D0E896F120055
:104B20003A0E8D6F830E8C6F120E8B6F6E0E8A6F26
:104B3000980E896F1200350E8D6F860E8C6F370EB2
:104B40008B6FBD0E8A6F060E896F1200300E8D6F4F
:104B5000890E8C6F700E8B6F5F0E8A6F410E896F9E
:104B600012002B0E8D6F8C0E8C6FBC0E8B6FCC0ECB
:104B70008A6F090E896F12006CDFFFEF22F071DF80
:104B8000FFEF22F076DFFFEF22F07BDFFFEF22F076
:104B900081DFFFEF22F087DFFFEF22F05ADF7FEFA8
:104BA00023F05FDF7FEF23F064DF7FEF23F069DF27
:104BB0007FEF23F06FDF7FEF23F075DF7FEF23F0D0
:104BC0001AEC21F003E18DEC2AF012003CEC1FF00E
:104BD00001013F0E176F800E166F136B146B156B70
:104BE000000128DFBCEC23F0CBEC1FF01BEC1FF026
:104BF00021DFC2EC23F0D6EC1FF05DEC1FF07EEC61
:104C00001FF07FEC23F0CBEC1FF0E1EC1FF03CEC4D
:104C10001FF0280E646F47EC1FF014DFC2EC23F086
:104C2000C0EC1FF05DEC1FF094EC1FF0FFEC22F0E5
:104C300094EC1FF0FFEC22F0CBEC1FF052EC1FF0D5
:104C40007FEC23F010EC1FF0C2EC23F010EC1FF00F
:104C50008D51885D0BE18C51875D08E18B51865D3C
:104C600005E18A51855D02E18951845D05E0644F6B
:104C700003D03CEC1FF0CFD7E5DEFFEF22F00101BF
:104C8000276B000129EC25F048D806E3CEEC25F08F
:104C90000101272B0001F6D793DFC1DE7FEC23F063
:104CA000EFEC1EF027C16AF06A5306E085EC21F0B4
:104CB000F4EC22F0C2EC23F012007ED873AF14D0D3
:104CC00078AF29D05AD87351785D0BE17251775D76
:104CD00008E17151765D05E17051755D02E16F513A
:104CE000745DD8B016D017D073BF02D078BF11D082
:104CF00044D87351785D0BE17251775D08E17151D1
:104D0000765D05E17051755D02E16F51745DD8B05B
:104D100002D0D89001D0D88012004ED873AF14D0F2
:104D200078AF29D02AD87351785D0BE17251775D45
:104D300008E17151765D05E17051755D02E16F51D9
:104D4000745DD8B016D017D073BF02D078BF11D021
:104D500014D87351785D0BE17251775D08E17151A0
:104D6000765D05E17051755D02E16F51745DD8B0FB
:104D700002D0D88001D0D89012001AEC21F003E1C3
:104D8000FDEC1EF00FD0D8901EEC20F0D8907233BE
:104D9000713370336F33728F1FEC21F003E104EC39
:104DA0001FF009D0D89018EC20F0D89077337633E4
:104DB00075337433778F120084C06FF085C070F044
:104DC00086C071F087C072F088C073F089C074F03B
:104DD0008AC075F08BC076F08CC077F08DC078F00B
:104DE000120002D8F7EF1FF033EC2AF037D8050E87
:104DF000616F00EE74F020EE65F0F0EC1EF010EE46
:104E00006FF0050E626F61C063F062516327630744
:104E10006307EF50E602F350DE26D9CF8EF0DACFEB
:104E20008FF0F450DE22E86ADE22632FFCD78EC0BA
:104E3000D9FF8FC0DAFF622FE6D7EE5220EE65F081
:104E4000060E636F6151635FDE52632FFDD7612FE2
:104E5000D6D740EC2AF091B30BD81200919373AFE0
:104E600002D015D8917378AF02D020D89173120078
:104E7000651F661F671F681F691F652BD8B4662BE7
:104E8000D8B4672BD8B4682BD8B4692B12006F1F25
:104E9000701F711F721F731F6F2BD8B4702BD8B483
:104EA000712BD8B4722BD8B4732B1200741F751FDA
:104EB000761F771F781F742BD8B4752BD8B4762B38
:104EC000D8B4772BD8B4782B1200C8DF33EC2AF093
:104ED000F0EC1EF0050E616F00EE74F0EE6605D08A
:104EE000612FFCD740EC2AF01200616B612BD89047
:104EF00078BF1CD074377537763777377837785165
:104F0000735D0BE17751725D08E17651715D05E1EA
:104F10007551705D02E174516F5DE8E2F0EC1EF0D6
:104F2000D890783377337633753374337851735D33
:104F30000BE17751725D08E17651715D05E17551C4
:104F4000705D02E174516F5D0AE374516F5F7551DA
:104F5000705B7651715B7751725B7851735B37ECA4
:104F600020F0612FDDD777DF6FC074F070C075F06F
:104F700071C076F072C077F073C078F0F7EC1FF074
:104F800040EF2AF0290E616FF0EC1EF07851735D4E
:104F90000BE17751725D08E17651715D05E1755164
:104FA000705D02E174516F5D0BE374516F5F755179
:104FB000705B7651715B7751725B7851735BD8800F
:104FC00030EC20F0D8901EEC20F07851735D0BE1AE
:104FD0007751725D08E17651715D05E17551705D43
:104FE00002E174516F5D0BE374516F5F7551705B3B
:104FF0007651715B7751725B7851735BD880612F0A
:10500000DFD7120033EC2AF0919373AF02D03FDF69
:105010009183F0EC1EF0280E616F0A0E626F00EEB5
:1050200065F0EF500F0B636F050E635DD8A002D0E3
:10503000030EEF26EF50F00B636F500E635DD8A0A8
:1050400002D0300EEF26EC52622FEBD7D8901EEC38
:1050500020F030EC20F0612FE0D740EC2AF0120075
:1050600050EC2AF015E268EC2AF01CE22FD844D864
:105070005AD892951200030E8E6509D08F678E2B39
:1050800091B58E2B030E8E5F8E5195EC12F01200AF
:10509000F2DF000EF86E3D0EF76E9E0EF66EAFEC70
:1050A00012F01200E8DF000EF86E3D0EF76EA20E51
:1050B000F66EAFEC12F0120050EC2AF0E9E268EC68
:1050C0002AF0F0E203D82FD89295120033EC2AF0A0
:1050D00000EE6EF011EE31F00A0E636FEDCF61F06D
:1050E0006139626F56D861C062F053D8632FF6D72A
:1050F000E76A40EC2AF0120033EC2AF08F5310E0FC
:1051000001EE44F011EE44F0140E616F8FC062F0B6
:10511000E5506107622FFCD7E5CFEDFF612FFCD78B
:1051200040EC2AF0120033EC2AF00A0E626F8F5125
:1051300062278E51625DD8B002D062C08EF08E516F
:105140008F5DD8A003D08FC08EF08E2B8F518E5FD5
:105150008E07090E616F8E51615F01EE31F0615370
:1051600004E0EECFE8FF612FFCD791A505D02B0E10
:1051700091BF2D0E08EC29F0918119D8919113D887
:105180008F5304E02C0E08EC29F009D840EC2AF0EB
:10519000120062510F0B3009E8CFE6FF12008FC0FA
:1051A00063F0929706D0010E636F929702D08EC083
:1051B00063F0635326E091A106D0EFCF61F0300E8B
:1051C000615DD8A4919192A711D063C06FF0020ED7
:1051D0006F6302D002EC29F0050E6F6302D002EC7F
:1051E00029F0080E6F6302D002EC29F0EECFE8FF41
:1051F00091B103D008EC29F002D004EC29F0632F20
:10520000DAD71200200E04D0200E92B5300E00D056
:1052100008EC12F0120033EC2AF00A0E616F8F5185
:10522000615F00EE65F0EF50614F0CD0EF50614FC1
:1052300002D0EE52F8D7EE526F6F490E6F6509D06B
:10524000010E06D00F0B6F6F040E6F6502D0100EAB
:10525000EF260A0E616F00EE65F0EF500700EE6E6C
:10526000E86AEF22612FF9D740EC2AF0120033EC04
:105270002AF0050E616F0A0E626F00EE6EF0EDCF40
:105280006FF06F51F00B07E162076F510F0B03E1F5
:105290006207612FF4D762C06FF0625140EC2AF0D0
:1052A000120097EC2AF0F0EC1EF002EC28F065C03A
:1052B0006AF066C06BF067C06CF068C06DF069C0E2
:1052C0006EF0050E8E6F8F6B9195929591999297D6
:1052D000120050EC2AF044E268EC2AF041E2D3ECF0
:1052E00022F0C8EC20F065C000F166C001F167C093
:1052F00002F168C003F169C004F16AC06FF06BC0CD
:1053000070F06CC071F06DC072F06EC073F002ECA2
:1053100028F065C007F166C008F167C009F168C0F0
:105320000AF169C00BF100C16FF001C170F002C158
:1053300071F003C172F004C173F060EC20F007C19A
:105340006AF008C16BF009C16CF00AC16DF00BC1C5
:105350006EF0140E8E6F0A0E8F6F91999297929540
:10536000919512003CEC1FF0906B889F1AEC21F095
:1053700014E029EC25F08DEC26F001E004E3CEECFE
:1053800025F0902BF6D71AEC25F05DEC26F005E021
:1053900004E3BCEC25F09007F6D769EC29F01BEC90
:1053A0001FF088BF918F0B0E8E6F0A0E8F6F918545
:1053B000919912005CEC28F0650E08EC29F0919FA1
:1053C00090BF918F90BF906DFDEC1EF090C06FF07C
:1053D00051EC29F091854BDF6FC08EF05CEC28F02A
:1053E000120047EC1FF010EC1FF0BCEC23F0ECECCB
:1053F0001FF073EC1FF068EC1FF0BCEC23F031ECF5
:105400001FF027C184F028C185F029C186F02AC188
:1054100087F02BC188F07FEC23F0ECEC1FF089ECD7
:105420001FF068EC1FF0BCEC23F0AAEC1FF0FFECBF
:1054300022F010EC1FF0C2EC23F0120033EC2AF043
:10544000FDEC1EF0050E616F10EE65F020EE6FF0C2
:10545000E6500F0BDF6EE638F00BDE12612FF8D747
:1054600040EC2AF01200E9CF45F1EACF46F1E1CF56
:1054700047F1E2CF48F1D9CF49F1DACF4AF1120032
:1054800045C1E9FF46C1EAFF47C1E1FF48C1E2FF6C
:1054900049C1D9FF4AC1DAFF1200DEEC22F003D085
:1054A000D3EC22F000D0839F7F0E83630CD0800E5C
:1054B000826307D0816705D0806703D07F6701D002
:1054C00002D0D88001D0D8901200DEEC22F003D0B8
:1054D000D3EC22F000D0839F7F0E83630BD0800E2D
:1054E000826308D0816706D0806704D07F6702D0CE
:1054F000D88001D0D890120002D8E9EF22F005D868
:10550000838F120002D8E9EF22F07F0E836F800EA6
:10551000826F7F6B806B816B120002D8E9EF22F003
:105520007F0E836F7F69806981698269120002D86A
:10553000E9EF22F07F6B806B816B826B836B1200D3
:10554000410E8D6FA00E8C6F896B8A6B8B6B120076
:10555000A0EC2AF07FEC23F0BCEC24F03CEC1FF034
:105560001AEC25F0C2EC23F0C0EC1FF01BEC1FF08E
:105570001AEC25F0BCEC23F031EC1FF047EC1FF0E7
:105580007FEC23F012004BC184F04CC185F04DC17B
:1055900086F04EC187F04FC188F0CEEC25F0BCEC10
:1055A00024F084C055F185C056F186C057F187C0FC
:1055B00058F188C059F1120055C184F056C185F0E8
:1055C00057C186F058C187F059C188F0D4EC25F056
:1055D000FCEC24F0FFEC22F02BEC24F084C060F112
:1055E00085C061F186C062F187C063F188C064F153
:1055F000120060C184F061C185F062C186F063C1B0
:1056000087F064C188F00101010E656F00019BEC19
:1056100025F05DEC26F009E30101040E656F000141
:10562000CBEC25F0C2EC25F018D090EC25F05DEC29
:1056300026F007E30101030E656F0001CBEC25F0B6
:105640000CD01AEC25F05DEC26F007E30101020E08
:10565000656F0001C2EC25F000D084C05BF185C00D
:105660005CF186C05DF187C05EF188C05FF1120019
:1056700055C184F056C185F057C186F058C187F0F6
:1056800059C188F00101030E5A6F0001B1EC25F0F9
:105690005DEC26F00BE3CBEC25F0CBEC25F0C2EC77
:1056A00025F00101080E5A6F00014CD0A6EC25F040
:1056B0005DEC26F009E3CBEC25F0CBEC25F0010105
:1056C000070E5A6F00013ED09BEC25F05DEC26F0F2
:1056D00009E3CBEC25F0C2EC25F00101060E5A6F70
:1056E000000130D090EC25F05DEC26F007E3CBEC28
:1056F00025F00101050E5A6F000124D01AEC25F0A7
:105700005DEC26F007E3C2EC25F00101040E5A6FB0
:10571000000118D053EC25F08DEC26F007E3DDEC0A
:1057200025F00101010E5A6F00010CD039EC25F073
:105730008DEC26F007E3D4EC25F00101020E5A6F40
:10574000000100D084C050F185C051F186C052F1F3
:1057500087C053F188C054F1120050C184F051C188
:1057600085F052C186F053C187F054C188F069ECCE
:1057700029F0050E8E6F010E8F6F29EC25F05DEC80
:1057800026F003E3040E8F6F0FD031EC25F05DECB3
:1057900026F003E3030E8F6F07D039EC25F05DECA4
:1057A00026F002E3020E8F6F0BEC29F065D85CEC5B
:1057B00028F05AC16FF0030E6F6309D0000EF86E27
:1057C0003D0EF76EA60EF66EAFEC12F054D0040E3E
:1057D0006F6309D0000EF86E3D0EF76EAA0EF66EDE
:1057E000AFEC12F048D0050E6F6309D0000EF86ED2
:1057F0003D0EF76EAE0EF66EAFEC12F03CD0060E1C
:105800006F6309D0000EF86E3D0EF76EB20EF66EA5
:10581000AFEC12F030D0070E6F6309D0000EF86EB7
:105820003D0EF76EB60EF66EAFEC12F024D0020EFF
:105830006F6309D0000EF86E3D0EF76EBE0EF66E69
:10584000AFEC12F018D0010E6F6309D0000EF86EA5
:105850003D0EF76EC20EF66EAFEC12F00CD0080ED5
:105860006F6309D0000EF86E3D0EF76EBA0EF66E3D
:10587000AFEC12F000D0120037EC29F0030E6F6588
:1058800002D0010E8F6F030E6F6302D0020E8F6F76
:10589000020E6F6302D0030E8F6F010E6F6302D092
:1058A000040E8F6F000E6F6302D0040E8F6F120014
:1058B0005BC184F05CC185F05DC186F05EC187F09C
:1058C0005FC188F069EC29F0060E8E6F010E8F6FB4
:1058D00039EC25F05DEC26F002E3020E8F6F31EC1F
:1058E00025F05DEC26F002E3030E8F6F29EC25F026
:1058F0005DEC26F002E3040E8F6F0BEC29F0BCDFA9
:105900005CEC28F065C16FF0010E6F6309D0000EEA
:10591000F86E3D0EF76EC60EF66EAFEC12F024D0A8
:10592000020E6F6309D0000EF86E3D0EF76ECA0EC0
:10593000F66EAFEC12F018D0030E6F6309D0000EB4
:10594000F86E3D0EF76ECE0EF66EAFEC12F00CD088
:10595000040E6F6309D0000EF86E3D0EF76ED20E86
:10596000F66EAFEC12F000D012004BC184F04CC1C7
:1059700085F04DC186F04EC187F04FC188F069ECCB
:1059800029F0050E8E6F020E8F6F0BEC29F037ECAD
:1059900029F0030E6F6104D0040E8E6F020E8F6F1C
:1059A000020E6F6504D0040E8E6F010E8F6F91850D
:1059B0005CEC28F0000EF86E3D0EF76ED60EF66E1B
:1059C000AFEC12F012004BC184F04CC185F04DC118
:1059D00086F04EC187F04FC188F069EC29F0040EC3
:1059E0008E6F010E8F6F0BEC29F037EC29F0030E50
:1059F0006F6104D0030E8E6F010E8F6F020E6F6504
:105A000004D0040E8E6F000E8F6F91855CEC28F031
:105A1000000EF86E3D0EF76ED60EF66EAFEC12F07D
:105A2000120050C184F051C185F052C186F053C1BB
:105A300087F054C188F069EC29F0040E8E6F010ED6
:105A40008F6F29EC25F05DEC26F003E3030E8F6FDA
:105A50000FD031EC25F05DEC26F003E3020E8F6FE2
:105A600007D039EC25F05DEC26F002E3010E8F6FD4
:105A70000BEC29F065D85CEC28F05AC16FF0030EEE
:105A80006F6309D0000EF86E3D0EF76EA60EF66E2F
:105A9000AFEC12F054D0040E6F6309D0000EF86E14
:105AA0003D0EF76EAA0EF66EAFEC12F048D0050E62
:105AB0006F6309D0000EF86E3D0EF76EAE0EF66EF7
:105AC000AFEC12F03CD0060E6F6309D0000EF86EFA
:105AD0003D0EF76EB20EF66EAFEC12F030D0070E40
:105AE0006F6309D0000EF86E3D0EF76EB60EF66EBF
:105AF000AFEC12F024D0020E6F6309D0000EF86EE6
:105B00003D0EF76EBE0EF66EAFEC12F018D0010E21
:105B10006F6309D0000EF86E3D0EF76EC20EF66E82
:105B2000AFEC12F00CD0080E6F6309D0000EF86EC7
:105B30003D0EF76EBA0EF66EAFEC12F000D012000A
:105B400037EC29F0030E6F6504D0050E8E6F000E42
:105B50008F6F030E6F6302D0010E8F6F020E6F63A3
:105B600002D0020E8F6F010E6F6302D0030E8F6F93
:105B7000000E6F6302D0030E8F6F120050C184F0CD
:105B800051C185F052C186F053C187F054C188F0ED
:105B900069EC29F0030E8E6F010E8F6F29EC25F052
:105BA0005DEC26F003E3020E8F6F11D031EC25F08F
:105BB0005DEC26F003E3010E8F6F09D039EC25F080
:105BC0005DEC26F004E3000E8F6F040E8E6F0BEC7D
:105BD00029F065D85CEC28F05AC16FF0030E6F63B2
:105BE00009D0000EF86E3D0EF76EA60EF66EAFEC05
:105BF00012F054D0040E6F6309D0000EF86E3D0E03
:105C0000F76EAA0EF66EAFEC12F048D0050E6F6379
:105C100009D0000EF86E3D0EF76EAE0EF66EAFECCC
:105C200012F03CD0060E6F6309D0000EF86E3D0EE8
:105C3000F76EB20EF66EAFEC12F030D0070E6F6357
:105C400009D0000EF86E3D0EF76EB60EF66EAFEC94
:105C500012F024D0020E6F6309D0000EF86E3D0ED4
:105C6000F76EBE0EF66EAFEC12F018D0010E6F6339
:105C700009D0000EF86E3D0EF76EC20EF66EAFEC58
:105C800012F00CD0080E6F6309D0000EF86E3D0EB6
:105C9000F76EBA0EF66EAFEC12F000D0120037ECD1
:105CA00029F0030E6F6504D0040E8E6F000E8F6F07
:105CB000030E6F6304D0040E8E6F000E8F6F020E02
:105CC0006F6302D0010E8F6F010E6F6302D0020E60
:0E5CD0008F6F000E6F6302D0020E8F6F1200F6
:020000040030CA
:0300010022193C85
:020005003D803C
:0200000400F00A
:10000000C2118DBF3CA7E8267FC2C1C0C0C03C91D1
:0E001000909080C2812602F941010100250076
:00000001FF
